:0200000270008C
:10800000807F002015D507003DD507003FD507002C
:1080100041D5070043D5070045D507000000000003
:1080200000000000000000000000000047D507002D
:1080300049D50700000000004BD507004DD50700CB
:108040004FD507004FD507004FD507004FD5070084
:108050004FD507004FD507004FD507004FD5070074
:108060004FD507004FD507004FD507004FD5070064
:108070004FD50700F1A007004FD507004FD50700E7
:108080004FD50700999207004FD507004FD507003D
:10809000559307004FD50700E1B007004FD5070003
:1080A0004FD507004FD507004FD507004FD5070024
:1080B0004FD507004FD5070000000000000000006A
:1080C0004FD507004FD507004FD507004FD5070004
:1080D0004FD507004FD507004FD50700000000001F
:1080E0000000000000000000000000000000000090
:1080F0000000000000000000000000000000000080
:10810000000000000000000000000000000000006F
:10811000000000000000000000000000000000005F
:1084000010B5054C237833B9044B13B10448AFF3CE
:1084100000800123237010BD8C2C00200000000080
:1084200054DA07000C4B43B10C480D4910B5AFF3BB
:1084300000800C48036823B910BD0A48036833B9AB
:108440007047094B002BF7D0BDE810401847064B8A
:10845000002BF5D0184700BF0000000054DA0700D9
:10846000902C0020702C002000000000154B002BE9
:1084700008BF134B9D46A3F5803A00218B460F465B
:108480001348144A121A00F063F80F4B002B00D067
:1084900098470E4B002B00D0984700200021040085
:1084A0000D000D48002802D00C48AFF3008000F00A
:1084B0002BF82000290000F069FD00F011F800BF42
:1084C00000000800807F0020000000000000000085
:1084D0008C2C0020BC3800200000000000000000B0
:1084E00008B5074B044613B10021AFF30080054BDC
:1084F0001868836A03B19847204600F031F800BF3E
:1085000000000000B4D5070070B50D4E0D4CA41B43
:10851000A4100025A54209D10B4E0C4C05F03EF8E5
:10852000A41BA4100025A54205D170BD56F8253026
:1085300098470135EEE756F8253098470135F2E7C0
:10854000682C0020682C0020682C00206C2C002057
:1085500002440346934200D1704703F8011BF9E738
:10856000FEE700BF024A1368013B1360704700BF7B
:10857000E830002030B50C490C4C8A6B85B0684659
:108580005C3103F05FFB9DE80F0084E80F00084BAF
:10859000E360084B084900221A605A602046074AE7
:1085A00003F0EAFD05B030BD043600205C32002047
:1085B000E9850700D02C002088D60700F030002085
:1085C00008B503F047F8BFF34F8F0549054BCA685C
:1085D00002F4E0621343CB60BFF34F8F00BFFDE7AF
:1085E00000ED00E00400FA055B689A68054B9A42CA
:1085F00006D14268836804490132013B0A604B603E
:10860000704700BF0CD60700D02C002070B50120A9
:1086100002F046FE0546B8B9114B124C1860A36B28
:1086200026468BB1FFF7A6FF70B1236A73B9A36921
:1086300063B10D4A13600C4B0C4A1868002103F01B
:1086400047F90B4B01221A70284670BDF36A002BC4
:10865000FAD1B369002BF7D0034B726A1A60EAE7CC
:10866000E830002004360020E0300020E430002014
:10867000EC3000202DE9F74F0B78012B0D46164604
:1086800001D0062B04D12A79012A0AD1A0490A7007
:108690009F4A1278012A08D0022A00F02C81052472
:1086A00022E0022AF2D007241EE0013B052B00F253
:1086B0004883DFE813F00600230043001D00460353
:1086C0001701AB6823B3B3F5807F00F2E580002487
:1086D000904B91481C7020222146FFF739FF8F4BA9
:1086E0001C63AA689A630124204603B0BDE8F08F9A
:1086F0008A4BDA6B72601B6CB360F4E7874CAA6834
:10870000E06BA36B1118994204D97060236CB360BD
:108710000324E9E75C306968204404F034FFAA6868
:10872000E36B1344E36304F14002A968686801F055
:10873000D7F8E36B20647360236CDDE7774FF96B48
:10874000BA6B914240F01981724D2B78002BCAD13F
:10875000FFF710FF0128A2D1714B93F874201C463B
:10876000002A00F0BA8093F87A30002B97D06D4E33
:1087700096E80600A9B1A2B194F8DB3013B194F8E1
:10878000DC3073B994F884305BB1D4F88830342B82
:1087900007D194F88CE06448002343F20C0C734535
:1087A00001DB0A24A0E7BCF8008050F8049FC14513
:1087B00000F0C9820133F2E794F87C30002BF0D04E
:1087C000B868D4F880308342EBD394F8E830002BBB
:1087D000E7D1564B3360202373600520514B01F0E5
:1087E00079FA0028DDD194F8E960514F51493246B9
:1087F000384604F0C8FE504B4A4A50491F600420D6
:108800005E6001F04FFA00287FF449AF4C4B94F8BA
:10881000A1201860032AC4D8DFE802F011403248D2
:1088200094F87C000028BCD0F868002BC9D0023B2B
:10883000012BCAD8D4F880308342B2D9C5E794F866
:10884000B020002AADD0D4F8B4201A603D4A374E8B
:1088500002F1200710685168344603C40832BA4256
:108860002646F7D1186800283FF452AF364A002157
:1088700003F02EF880B9012402F066FE2C7033E775
:1088800094F8A820002A8CD0D4F8AC1019602F4A94
:10889000C2F5FC229142D9D9042425E794F8A220FC
:1088A000002A3FF47EAFD4F8A420CEE794F8A820A5
:1088B000002A3FF476AF94F8A220002A3FF471AF6B
:1088C000D4F8A420D4F8AC1050181860002A3FF453
:1088D0001FAF00293FF41CAFD9E71B78002B3FF4F2
:1088E000DEAE5EE70D4B1A6CB260DB6B73604FF46B
:1088F00080733360F7E6013B052B00F22282DFE84C
:1089000013F02700690032012D012002180200BF78
:10891000602C0020EC3000203C3600200436002083
:10892000F0300020D02C00207C310020B02C002022
:108930001C320020DA310020A82C002034D7070098
:10894000E0300020AB310020E43000200080070040
:10895000AB68002B3FF4DCAEC3F30B023AB18E4A96
:108960008E49526D09681A448A427FF4D1AEB3F53C
:10897000805F91D88A4A12780AB90824B4E6864AF8
:108980008649506D096803448B42F6D8D36C9364D2
:10899000AB68536410651063824A834C1378A968EE
:1089A000013303F003031370804B00221A80236805
:1089B0007F4A013323607F4B1B6801F6FF71090B6F
:1089C000184402F0CDFC00283FF48DAE2368013B33
:1089D000236064E6704C236D7360A36CB360704BCE
:1089E0001B78002BC9D0A968B1F5807F3FF654AF42
:1089F000626D236D9B1A626C0B4493423FF688AE06
:108A000004F148026868694FDFF89881DFF8A8A18F
:108A100000F066FFA064AA68236D134423657360A9
:108A2000A36CB360AA683B889918FF29696839D894
:108A300098F80000019303EB0020504404F0A3FDDC
:108A4000A868019B184438803A88002A3FF44BAE4E
:108A5000636D206B616CD31A03448B42FFF443AE09
:108A6000544B514DD3F800E02B6898F800C05249A0
:108A7000013303322B6092104D4B01EB0C217044FB
:108A800002F026FC00285ED1236B3A88134423634E
:108A900098F80030013303F0030388F80030002316
:108AA0003B8020E698F80090C3F5807B4FEA0929C7
:108AB0001FFA8BFB03EB09005A46504404F063FD98
:108AC0004FF480733B80AB68A3EB0B03AB606B6828
:108AD0005B446B60DFF8D0B0364B206BD3F800E01E
:108AE000DBF800300133CBF800304022304B0AEB8A
:108AF0000901704402F0ECFBC0B9236B3A881344BF
:108B0000236398F80030002201333A80AA6803F00A
:108B1000030388F80030002A96D02748696800EBE4
:108B2000032004F030FDAB683B808DE7DBF80030BC
:108B3000013BCBF80030E36CA364636D2365736085
:108B4000E36CB360DDE72B68013B2B60E36CA3644F
:108B5000636D23657360E36CB36099E70E4B1A6D28
:108B600072609B6CC8E50C4D2A6D6B6D696CD31AF5
:108B700099427FF402AFAB6C6A650020EB646864D5
:108B800002F0E2FC054B296D1A68914298467FF489
:108B9000AAAD054C14E000BF04360020E0300020F0
:108BA000EC300020D82C0020E8300020DC30002001
:108BB00065850700E4300020DC2C002002F012FB69
:108BC0002368002BFAD16B4E96F8B930032B2CD1C9
:108BD000694F6A496A4B3B604FF020093B46D8F821
:108BE00000200968C7F80490052001F073F84A4690
:108BF000002806F1BB01386814BF0A24012404F0E0
:108C0000B3FC002818BF05246B6983B1012B7FF4E6
:108C1000C8AD5C4B012C40F0888096F8A120032A57
:108C200079D8DFE802F0060C6C720A24ECE7564BA8
:108C3000F0E701229A60D6F88020AA6004E0A5221D
:108C40009A60D6F8A4206A63AA6C5A60D8F800200B
:108C50001A60002120224D484D4E4E4FFFF778FC00
:108C6000B222FF214C48FFF773FC00232B634B4DCE
:108C7000284602F069FC11287FF436AD484B326873
:108C800000BF00BF00BF00BF00BF00BF00BF00BFEC
:108C9000BA422FD000BF00BF00BF00BF00BF00BF5F
:108CA00000BF00BF00BF00BF00BF00BF00BF00BFCC
:108CB00000BF00BF00BF00BF00BF00BF00BF00BFBC
:108CC00000BF00BF00BF00BF00BF00BF00BF00BFAC
:108CD00000BF00BF00BF00BF00BF00BF00BF00BF9C
:108CE00000BF00BF00BF00BF00BF00BF00BF00BF8C
:108CF00000BF00BF013BC3D102F074FAB8E7AA225B
:108D00009A60D6F88020EA609EE7AC229A60D6F896
:108D1000A4206A63F5E722B1023A012A03D80A24A3
:108D2000EFE70A2487E70A248EE700229A605A6058
:108D30008EE71C4B9A6CB2601B6D73604FF48053CE
:108D4000D7E50224D0E494F8A130032B3FF629ADF7
:108D500001A050F823F000BFB9870700698D070014
:108D60002188070021880700023B012B3FF62DAD2B
:108D700000205FE5F0300020D02C0020E4300020FF
:108D8000B02C0020283600201C3600203C36002065
:108D9000642C00200024F40060360020C185070008
:108DA000A08601000436002070477047BFF34F8F44
:108DB0000549064BCA6802F4E0621343CB60BFF377
:108DC0004F8F00BFFDE700BF00ED00E00400FA0593
:108DD0004FF0A043D3F81005054B93F8972093F874
:108DE0009630D040DB0648BFC04300F0010070471A
:108DF000ACD7070008B5FFF7D9FF08B5FFF7D6FFD6
:108E00000D4B00EB80001A1870B51B5C5478C3F34F
:108E100000134FF0A04204F5E07599424FF00306AD
:108E20004FF0010342F8256003FA04F30CBFC2F8C7
:108E30000C35C2F8083570BDACD70700022808B55C
:108E40000BD003280BD078B90848FFF7AEFF0121FB
:108E50000C20BDE80840FFF7D3BF0548F5E70548FB
:108E6000BDE80840FFF7A1BF08BD00BF3CD7070021
:108E700051D707004ED707002DE9F843FFF7A8FFA9
:108E80000546E8B1FFF790FF39483A4FDFF8F48024
:108E9000DFF8F490FFF789FF3748FFF786FF374880
:108EA000FFF783FF40F6B834FFF792FF064600282D
:108EB00057D044B9264601210C20FFF7A1FF3546C3
:108EC0002846BDE8F88340F2E7333A6800BF00BFA8
:108ED00000BF00BF00BF00BF00BF00BF42452FD092
:108EE00000BF00BF00BF00BF00BF00BF00BF00BF8A
:108EF00000BF00BF00BF00BF00BF00BF00BF00BF7A
:108F000000BF00BF00BF00BF00BF00BF00BF00BF69
:108F100000BF00BF00BF00BF00BF00BF00BF00BF59
:108F200000BF00BF00BF00BF00BF00BF00BF00BF49
:108F300000BF00BF00BF00BF00BF00BF00BF00BF39
:108F4000013BC3D114F0030F0CBF012100210C2001
:108F5000FFF756FF630602D14846FFF726FF013CA4
:108F6000A2E7002CA7D00648FFF71FFF2E46A2E776
:108F70005DD70700642C00206AD7070081D707005F
:108F80009CD707000024F4009AD70700002110B5F1
:108F90000C20FFF735FF104B93F8972093F896308D
:108FA000DB0647BF03210B46022301211B0443EAD2
:108FB000810302F5E0724FF0A04141F8223002F047
:108FC000D7F8044608B1FFF7F1FE43F2080318682A
:108FD00002F0F2F8204610BDACD7070012F00303F0
:108FE00010B511D1094C22604C1CE400A4B22244FB
:108FF000074C2260074A1370074A1370074A108013
:10900000074A1180184610BD072010BD7432002099
:10901000703200206C3200207C3200207832002038
:109020007A3200202DE9F743284D2B888B420646E3
:109030000C46174646D302A84FF0000800F8018DF1
:1090400000F014FC224B234A18781178CBB2224945
:1090500009888B4238BF0133C0B238BF5FFA83F84A
:10906000404528D092F800801378DBB2994286BF41
:109070000133DBB2002313709DF8070000F01AFCE7
:109080004FF6FF7398451FD0144B1B6803EBC809BC
:1090900043F8387096B18CB1114B28881B68224672
:1090A000314608FB003004F06EFAA9F804400020B5
:1090B00003B0BDE8F0834FF6FF78DDE70020A9F8A4
:1090C0000400F5E70920F3E70420F1E778320020F7
:1090D0007C3200206C3200207A3200207432002072
:1090E00070320020F8B5124C124D264622782B78AB
:1090F0009A4200D1F8BD23780F48104A07881268B9
:109100000F48DBB219B202EBC10E006852F83120F1
:10911000BEF8041003FB070090470A4A2378128820
:10912000DBB29A4286BF0133DBB200233370DDE746
:109130007C3200206C320020783200207432002013
:10914000703200207A32002010B50A494A788C78B3
:10915000531CDBB29C4208BF00230C789C421FBF0B
:109160000370486802EB420200EBC20008BF002017
:1091700010BD00BF8432002073B5054602A800244C
:1091800000F8014D0E4600F071FB0DF10600FFF7EF
:10919000DBFF90B106700A4B9DF8062045605A70BF
:1091A0009DF8070000F086FB24B9064B4FF48012AF
:1091B000C3F80021204602B070BD0424F0E700BFD0
:1091C0008432002000E100E0204B21491A682F235F
:1091D00000BF00BF00BF00BF00BF00BF00BF00BF97
:1091E0008A422FD000BF00BF00BF00BF00BF00BF3A
:1091F00000BF00BF00BF00BF00BF00BF00BF00BF77
:1092000000BF00BF00BF00BF00BF00BF00BF00BF66
:1092100000BF00BF00BF00BF00BF00BF00BF00BF56
:1092200000BF00BF00BF00BF00BF00BF00BF00BF46
:1092300000BF00BF00BF00BF00BF00BF00BF00BF36
:1092400000BF00BF013BC3D1704700BF642C0020AA
:109250000024F4000C4B0D484FF4003210B5C3F855
:10926000802001244FF48033C0F84833C0F808331D
:109270004460FFF7A9FF064B846000201860FFF7E9
:10928000A3FF044B187010BD00E100E00010014086
:109290009C3200208D3200202DE9F0412549264BDB
:1092A0000025C1F84051C1F84451C1F84851C1F8F6
:1092B0004C51C1F80051C1F804511B68002B31D04A
:1092C000D1F804451D49DFF888800968641A24F044
:1092D0007F442F461A68A2420FD8A41A15441A7C5C
:1092E000DE694AB1D8F800201F74FAB1996958694B
:1092F000904708B1FFF781FDB6B9114B114A1978B3
:1093000013788B4205D10133DBB2022B08BF002357
:10931000137012780C4B43F822500C4B4FF4801210
:10932000C3F80021BDE8F0813346D3E75A69986954
:109330009047E1E700100140A03200209C3200205D
:1093400098320020993200209032002000E100E0A5
:10935000803200202DE9F04F9A4A9B491378097812
:109360009A48994287B0076876D00133DBB2022B66
:1093700008BF002313701278954B53F822403B1915
:1093800023F07F43036001230293924BD0F800A0A7
:109390001A780192904AD2F800C05A7805925A6819
:1093A0009B7804938D4B03920020019A93F800E080
:1093B00081466346804605998A4250D1B8F1000F34
:1093C00002D0864D85F800E0B9F1000F02D07F4D44
:1093D000C5F800A0804D00B12B60029B002B6DD121
:1093E0002B68B3EB0C0318BF0123029300262B68F4
:1093F00005937A4B059893F800B0744B4FF0000C2E
:10940000D3F800806746E146002E00F0EE80334638
:10941000F6695C687249D3F808E0A4EB080525F00A
:109420007F458D4200F2A58075441D604FF001011B
:10943000C3F80490C3F808901974C3F81C9038B1AD
:109440001D680468A54200F2AD80651B0560D86107
:1094500018464FF0010CD7E70024029495E702EB81
:1094600042050499039E0132D2B28A4208BF00220B
:10947000039906EBC50611F83550022D09D0032DCE
:1094800099D1002B97D04FF0000119740120DB69AE
:10949000F7E775689B461E46BBF1000F8BD05D4514
:1094A00000F0FF805E46DBF81CB0F5E74D49012077
:1094B000886081469A4680468646F9E04FF0000E65
:1094C0002B6876467046F04623B9BEF1000F8ED069
:1094D0002B608CE7D3F800C0A44507D9BEF1000F7C
:1094E00000D02B60ACEB04041C6080E7A4EB0C0400
:1094F0006044D3F80CC0C3F80080D3F81C90BCF1D2
:10950000000F09D007EB000E2EF07F4EDE61C3F88E
:1095100004E0C3F808C01E464B46DDF808E0D3E778
:10952000019B039903EB430301EBC3040199013150
:10953000C9B20191019D0499A94208BF0025039970
:10954000019511F83350012D4ED163681F7C002F17
:109550004BD1A1685960E16899602169D96064695B
:109560009C61BBF1000F02D05F605F4651E72F4660
:109570004FE7A8EB040424F07F4474453ABFAEEBF8
:1095800004041C60C3F8009050E7A5EB0E05D4F866
:109590001CE0A246BEF1000F11D11D60C3F81CE013
:1095A000E36131E782460446D4F800E0AE45ECD3EF
:1095B000AEEB050EC4F800E0A6465446EDE774464F
:1095C000F2E700BF98320020993200209C32002040
:1095D0009032002084320020A03200208C32002003
:1095E000FEFF7F00001001400127019B9A4297D1A6
:1095F0000FB1354B1A70354BBCF1000F00D018601D
:109600001B68059A9A4202D1029A002A40D0002B88
:1096100044D02F482F4FD0F804651C683B78A6EB48
:10962000080525F07F45033582469BB94FF480330A
:10963000C0F84433C0F80433274B4FF400324FF0E6
:109640000109C3F880211A60C0F80090FFF7BCFD43
:1096500087F80090AC422CBFA044A84428F07F4378
:10966000CAF84035DAF80425921B22F07F429B1B92
:10967000033223F07F439A420AD9DAF80435CAF854
:109680004035FFF7A1FD144B4FF40032C3F8002121
:10969000124B00221A7007B0BDE8F08FFFF7DAFD19
:1096A000F6E7B54204D1DB69002B3FF4FFAE0120A1
:1096B000D5F800B0ED69F561002D3FF47CAE2E6861
:1096C0005E442E6077E600BF84320020A032002086
:1096D000001001408D32002000E100E08C320020BB
:1096E0002DE9F04112F0030406460F461546984650
:1096F00028D13AB3FFF7AEFD144B154A1C705C70CD
:109700009F705D60134BC2F800801C60124B1C7090
:10971000124B1C70124B4FF48012E021C3F88021D1
:1097200083F814131A6002F18042A2F56F222046DA
:10973000C2F8086583F811130A4BD2F804251A60A1
:10974000BDE8F0810720BDE8F08100BF8432002031
:1097500080320020A0320020983200209932002070
:1097600000E100E09C320020074B5B684BB132B156
:1097700028B10368187C20B959745A6170470720D2
:1097800070470820704700BF843200202DE9F7435E
:109790001E4F7B6805460E469046ABB3A0B3042926
:1097A00030D9436983B3437C02A80024012B00F81D
:1097B000014D0CBF8946A14600F058F80DF1060096
:1097C000FFF7C2FCE0B101230370114B4560D3F8F1
:1097D000043583609DF80630C660C0F81090C0F86C
:1097E00014807B709DF8070000F064F824B9094BE1
:1097F0004FF48012C3F80021204603B0BDE8F08387
:109800000424EFE70724F7E70824F5E78432002073
:109810000010014000E100E0064A52683AB130B160
:10982000426922B1002202740221FFF7A5BC082080
:10983000704700BF84320020082910B5044602D0CA
:109840000020FFF7DAFA23686068BDE81040184787
:1098500007B5054A8DE8030008216846FFF7E2FBDB
:1098600003B05DF804FB00BF3998070070B5EFF353
:10987000108672B60C4A946801239CB993600B4B16
:109880000B4DD3F8801029401160C3F88050D3F8F5
:10989000841051604FF0FF32C3F88420047006B981
:1098A00062B670BD0370FAE7A432002000E100E068
:1098B000FC06FFBC10B5084B9A685AB150B9EFF3DB
:1098C000108272B605491C680C605C684C60986038
:1098D00002B962B610BD00BFA432002000E100E072
:1098E00030B53AB11368DB430A4D0144814204D1DB
:1098F000D84330BD4FF0FF33F6E710F8012B53404B
:10990000082213F0010418BF2C46013A84EA5303DD
:10991000F7D1EBE72083B8EDF7B50D4617461E46A5
:109920000446B0B1A9B1A3B140EA01039A0712D12C
:10993000B30710D103F088FC334600903A4629461D
:10994000204603F085FC00280CBF0B20002003B04C
:10995000F0BD0E20FBE71020F9E729DF704728DF74
:1099600070470000084B5A6E013A5A6622B90749FF
:109970000A7822F002020A701A6E0132042A08BF25
:1099800000221A66704700BFB4320020B0320020B7
:1099900038B50C4C626E042A054611D0236E134470
:1099A000032B02F1010288BF043B6266182202FB0E
:1099B000034400212046FEF7CBFD2C60012038BD7A
:1099C000002038BDB432002030B5044685B00D46C5
:1099D000102200216846FEF7BBFD237A012B0AD036
:1099E000022B0ED063680193236829469B68684662
:1099F000984705B030BD23690293A38AADF80C30B7
:109A0000F0E70123A2898DF80030E389ADF80A2040
:109A1000D31AADF80830E5E738B51C4B5A6E194635
:109A2000002A32D01C6E182202FB04331A7A012A53
:109A300007D0022A23D018460921BDE83840FFF795
:109A4000C3BF1825D88A9A8A05FB0414121AE16844
:109A50002469B2F5806F4FEA80000144B4BF92B22E
:109A60004FF480622044FFF778FF11280BD1084A99
:109A7000137823F0020343F00403137038BD988970
:109A8000FFF76DFFF1E70028D5D138BDB4320020D3
:109A9000B0320020054A137813F0060F04D143F0CA
:109AA00002031370FFF7B8BF704700BFB032002049
:109AB000034A137843F0010313700020704700BF7E
:109AC000B0320020F7B51F461F4B1B781646DA0749
:109AD00004460D4629D528B11C4B984202D31C4B95
:109AE00098422CD302201EE05DB346EA05039B0793
:109AF0001DD123689D421CD3626805EB87039A42FF
:109B000017D3C7B101A8FFF743FFB0B1019B089A73
:109B10001C6001995A6001230B72CE600D618F8227
:109B2000FFF7B8FF002003B0F0BD0120FBE70620DF
:109B3000F9E70520F7E70420F5E70720F3E7002E13
:109B4000D2D10320EFE700BFB0320020742C0020F8
:109B5000842C0020F7B51F461D4B1B78DB070546FC
:109B60000C46164626D528B11A4B984202D31A4BFA
:109B7000984229D302201BE0C4F30B03E3B92B68FE
:109B80009C421BD36B6804EB0632934216D3BEB1E2
:109B900001A8FFF7FDFEA8B1019A82E8A000019B91
:109BA0000222240B1A729C811E82FFF773FF002091
:109BB00003B0F0BD0120FBE70620F9E70520F7E739
:109BC0000420F5E70720F3E70029D5D10320EFE7CC
:109BD000B0320020742C0020842C002038B52A4A92
:109BE00013780146980742D5284A146E1820022996
:109BF00000FB042005D003292DD0BDE83840FFF735
:109C00000BBF234B00211970037A012B0CD0022BC0
:109C1000F3D18389028A01338381C38901339BB2E3
:109C20009A42C381E9D111E0858AC38AE91AB1F564
:109C3000806FB4BF89B24FF480610B4418219BB28E
:109C400001FB04229D42D382D7D10021FFF7BCFE45
:109C5000FFF788FED1E70E4A13780133DBB2032BFE
:109C600001D81370C9E7002313700821EEE75907E4
:109C7000C3D50649496E03F0FB0313700029BCD01D
:109C800043F00203EDE700BFB0320020B432002001
:109C90001C330020024B586E031F58425841704736
:109CA000B4320020042810B40C4611460CD162686E
:109CB000402A0DD15A68402A0AD120681B685DF8F5
:109CC000044B06C9FFF728BE06205DF8044B704719
:109CD0000920FAE7F0B505289DB00E4617461C4648
:109CE00015D15D68202D14D1684600F0B1F860B937
:109CF0003A463146684600F0DBF830B90122216867
:109D0000684600F0F9F800B965601DB0F0BD0620A6
:109D1000FBE70920F9E700002DE9F04F0022C9B068
:109D20004B780C781B0443EA0463CC7823438C788B
:109D300043EA042308AC0431A3500432402AEFD193
:109D4000234638AD996B1E464FEAF14282EA7142D2
:109D500082EA9122716A366853F8044F31440A440A
:109D60004FEAB44181EAF41181EAD4010A449D42E8
:109D7000DA63E7D1036D0093436D0193836D029322
:109D8000C36D0393036E0493436E0593836E069332
:109D900004A991E80250C36EDDF80C80029DDFF843
:109DA000AC9007939DE850009B4600274FEAF123B3
:109DB00083EAB11383EA716A59F827301A4608AB6F
:109DC00053F827301A44134653442EEA010201EA9D
:109DD0000C0A82EA0A021A444FEA743A85EA060338
:109DE0005A448AEAB40A06EA050B234083EA0B03C5
:109DF0008AEAB45A01379A44402F02EB0803F3462B
:109E00005244A8461AD1009F1744019A076522447C
:109E10004265029A32448265039A2A44C265049AD2
:109E20001A44059B02660B444366069B63448366A3
:109E3000079B7344C36649B0BDE8F08FE6463546DC
:109E40008C46264619461446B0E700BF4CD807009A
:109E500030B5E0B10F4A02650F4A42650F4A82658C
:109E60000F4AC2650F4A02660F4A42660F4A82666F
:109E70000024002502F17452C0E91245A2F5230224
:109E80000023A2F692420364C266184630BD0E203B
:109E900030BD00BF67E6096A85AE67BB72F36E3CF2
:109EA0003AF54FA57F520E518C68059BABD9831FA5
:109EB000F8B50446F0B10AB90020F8BDD1B10D469D
:109EC0008E180027B542F7D0236C15F8012BE25409
:109ED0000133402B2364F5D121462046FFF71CFFB8
:109EE000D4E9120110F5007041F10001C4E912013A
:109EF0002764E7E70E20F8BD70B50D461646044608
:109F0000002800F08680002900F08380026C802108
:109F1000372A00EB020381544BD800F138020021AC
:109F200001339A4243D1D4E91223206C0821E1FB8A
:109F3000002322FA01F1C4E9122384F83F2084F8B7
:109F40003E10110C120E84F83C201A0A84F83B30A3
:109F500084F83A201A0C1B0E84F83D1084F839203E
:109F6000214684F838302046FFF7D6FE691E8EB3AE
:109F70000023E26EDA4001F8012FA26EDA400A7186
:109F8000626EDA400A72226EDA400A73E26DDA40DB
:109F90000A74A26DDA400A75626DDA400A76226DA3
:109FA000DA400833202B0A77E3D1002070BD197006
:109FB000B6E7002101331A1B3F2A09D92146204662
:109FC000FFF7AAFE382200212046FEF7C1FAAAE7D1
:109FD0001970EFE71823226DDA4001F8012F626D46
:109FE000DA400A71A26DDA400A72E26DDA400A7351
:109FF000226EDA400A74626EDA400A75A26EDA40A6
:10A000000A76E26EDA40083B13F1080F0A77E2D1D4
:10A01000CBE70E2070BD03685A681B689A422FBFB9
:10A02000D01A80680130801838BFC01A70470268A3
:10A030008168536810688B4234BF01330023C31A10
:10A04000584258417047F7B5044602A8002300F86B
:10A05000013D0D46FFF70AFC2046FFF7E8FF10B16F
:10A06000237C002B3CD12268A16853688B4234BF0B
:10A07000591C0021516038B12168A0680A688242E9
:10A0800034BF013200220A60E2686068511E07296D
:10A0900020D8DFE801F004101F141F1F1F182A78B2
:10A0A000C2542046FFF7B7FF23689A68904200D950
:10A0B0009860002415E02A8820F81320F1E72A6828
:10A0C00040F82320EDE7D5E9006700EBC300C0E9C5
:10A0D0000067E6E7294602FB030003F054FAE0E7D5
:10A0E00004249DF80700FFF7E5FB204603B0F0BD10
:10A0F00013B502A8002300F8063DFFF7B7FB00F0F8
:10A10000A3FFE0B9114B1A68CAB1114CD4F8082367
:10A11000D20714D518601B68019302A9019BD4F8DB
:10A12000083501F8053D0B48FFF78DFF0948FFF79B
:10A130007EFF20B1084A0123C4F8083313609DF85C
:10A140000200FFF7B7FB02B010BD00BF00D1004016
:10A1500000D000404CD9070004D000400B4B022235
:10A16000C3F80425D3F80024002AFBD0C3F808055F
:10A17000D3F80024002AFBD00022C3F80425034AA8
:10A18000D2F80034002BFBD0704700BF00E0014044
:10A190000F4B10B50124C3F80445D3F80044002C3C
:10A1A000FBD00B4B043900EB8202904207D1002216
:10A1B000C3F80425D3F80024002AFBD010BD51F8C1
:10A1C000044F40F8044BD3F80044002CFBD0ECE7DC
:10A1D00000E001406CDF70476DDF704772DF704751
:10A1E00073DF704774DF704776DF70477ADF704740
:10A1F0007CDF70477DDF70477FDF704786DF704709
:10A20000A0DF7047A2DF7047A5DF7047A6DF704769
:10A21000A8DF7047A9DF7047ADDF704763DF704785
:10A2200067DF704713DF704730B587B004460D46CF
:10A23000ADF806200021102202A8FEF789F90123BB
:10A240008DF80A300DF10603049302A9044BADF812
:10A25000085020460593FFF7D9FF07B030BD00BF77
:10A26000B4330020FEF7C9BD10B40D4B0246188868
:10A270004FF6FF7398420FD00A4B1B68DB070BD5D4
:10A28000094B60245A7099701C70084B5DF8044BA0
:10A2900099890322FFF7C8BF08205DF8044B704777
:10A2A000622C0020B0330020B43300209C33002007
:10A2B00010B5314C23685A075BD443F00402226086
:10A2C0002E4A2F4811682F4A00BF00BF00BF00BFB1
:10A2D00000BF00BF00BF00BF81422FD000BF00BF42
:10A2E00000BF00BF00BF00BF00BF00BF00BF00BF76
:10A2F00000BF00BF00BF00BF00BF00BF00BF00BF66
:10A3000000BF00BF00BF00BF00BF00BF00BF00BF55
:10A3100000BF00BF00BF00BF00BF00BF00BF00BF45
:10A3200000BF00BF00BF00BF00BF00BF00BF00BF35
:10A3300000BF00BF00BF00BF00BF00BF013AC3D1D4
:10A34000114A10884FF6FF72904204D01321FFF794
:10A350004BFF60B110BD9B0709D5FFF743FF48B91C
:10A360000120FEF76BFD236843F00203236000F039
:10A3700021FC002010BD00BFB0330020642C002061
:10A380000024F400C0D40100622C002030B52F4D11
:10A39000296811F002018BB056D1102201A8FEF7F6
:10A3A000D7F80B23ADF80230012202238DF81430C8
:10A3B0008DF815208DF81830062259238DF81620B7
:10A3C0008DF819300322FE230DF102010DF11D005D
:10A3D0008DF817208DF81A30FFF70CFF044640BBAC
:10A3E000BDF802100B2927D84B1C8DF81B30092310
:10A3F00019448DF81C3089B200231A46C9B205A849
:10A40000FFF7ECFE0446A0B98DF8040002908DF829
:10A410000C002823ADF8100001A8ADF80E30FFF7AE
:10A42000DFFE044628B9FEF709FD2B6843F002035E
:10A430002B6020460BB030BD0C238DF81B30082359
:10A440008DF81C301421D7E70024F2E7B033002048
:10A4500010B4154B024618884FF6FF7398421FD070
:10A46000124B1B68DB071BD5114B60241C700324A7
:10A470005C7001249C70140ADA701C71140C120EAA
:10A480009A710A0AD9711A720A0C090E5A729972D3
:10A490005C71084B5DF8044B99890B22FFF7C4BE31
:10A4A00008205DF8044B7047622C0020B033002078
:10A4B000B43300209C3300202DE9F041044688B0DD
:10A4C00000F07EFB2388142B00F03F8118D8102B5E
:10A4D00070D005D8022B00F0898008B0BDE8F0816B
:10A4E000112B76D0132BF8D19F4800231A468521D3
:10A4F0000088FFF781FE0028EFD0FEF77EFCECE736
:10A50000522B00F0298147D8502B00F03981512B74
:10A51000E3D1A579002DE0D0102200210DEB02003F
:10A52000FEF716F8022DD8D1904D2289AB899A42B8
:10A53000D3D1A37B043B022BCFD99DF816308A4E92
:10A54000298A3088CDF808D043F001038DF8163001
:10A55000238AADF81830638AADF81A3004F1140379
:10A560000222079300238DF810200193ADF80420F8
:10A5700001AAFFF749FEB04600283DD1684600F029
:10A5800075FB002838D140F2FD1304A93088ADF8DE
:10A590001430FFF73DFEA0E7552B00F01B81562B32
:10A5A0009BD1A379002B98D16F4B13211888FFF70B
:10A5B0001BFEA0E70120FEF741FC0220FEF73EFC57
:10A5C000694BA2881A806A4A136823F00203136059
:10A5D00083E70320FEF732FCFFF7D8FE08B1FEF751
:10A5E0000CFC614B4FF6FF721A8076E75E4B002140
:10A5F0001888FFF715FE7EE7002304A9B8F80000CD
:10A60000ADF81430FFF704FE00287FF466AF049025
:10A6100005900690019002900390207D431E052B2B
:10A6200000F29180DFE803F00329391E8F4C638A22
:10A63000062B04D003210120FFF716FE4DE74D4BFA
:10A640001A884D4B1A80637D029301A9D4F8163005
:10A650000393012404AA00208DF80440FEF70AF8B1
:10A660000146E8E7032301A904AA00208DF804307D
:10A67000FEF700F801460420DEE7638A032B02D0D0
:10A6800003210220D8E7A27D637D43EA0223394AF1
:10A690001380394A01211380F3E704230DEB0301F2
:10A6A00004AA00208DF80430FDF7E4FF01280146DC
:10A6B00004D106990598FFF7CBFE0EE70320BBE710
:10A6C000638A022B02D003210620B5E7637D029343
:10A6D00001A9062704AA00208DF80470FDF7CAFF1F
:10A6E00001280146F0D1B8F800004FF6FF739842F8
:10A6F0003FF4F3AE1E4B1B68DB077FF5EEAE1F4B3E
:10A70000049E059C9970310A1971310C069A597191
:10A71000210A1972210C5972110ADE70DC71360E91
:10A72000240EDA721973110C120E4FF0600E597369
:10A730009A739E719C720F22A98983F800E05F7062
:10A74000FFF772FDC9E6032176E700231A46194692
:10A75000A088FFF753FDCEE600231A461946A088CD
:10A76000FFF758FDC7E600BF622C00209C33002095
:10A77000B0330020C4330020C6330020B43300209F
:10A78000174BE2889B889A427FF4A7AE00200223F1
:10A7900001908DF8043004F11203029304AA238A75
:10A7A000039301A9049005900690FDF763FF0D4BFC
:10A7B0001D88002D3FF491AE0B4C2388013B9BB2CA
:10A7C0002380002B7FF489AE06990598FFF740FEA1
:10A7D000258082E61721A088FFF71EFD8BE600BFCB
:10A7E0009C330020C4330020C63300202DE9F047FD
:10A7F000074694B0002800F09E80504B4FF6FF7241
:10A8000014A91A804FF65963012021F8483D3A46B1
:10A810008DF80A00FFF7F4FC0446002840F087801A
:10A82000474B04AA03F110061546186859681446E8
:10A8300003C40833B3422246F7D1B91C2846FFF7B8
:10A84000EDFC0446002872D101461C224FF0140A88
:10A850000DA8FDF77DFE2146524608A8FDF778FEBB
:10A860009DF83430ADF8044043F004038DF83430E3
:10A87000BB788DF80E3002234FF00109ADF80C3093
:10A88000230AA04669F3030369F3420469F307133B
:10A89000E4B28DF8053044EA090401AD03AE3B1D76
:10A8A00008AA0DA938888DF8064008960995ADF8D4
:10A8B0002CA0FFF7A7FC0446002838D101461C2233
:10A8C0000DA8FDF745FE2146524608A8FDF740FEBB
:10A8D0009DF83430ADF8044043F018038DF834305F
:10A8E000BB788DF80E30434669F34203DBB243F088
:10A8F0001103240A8DF8063069F30304172369F362
:10A900000714ADF82C3008AA07F10C030DA93888FC
:10A910008DF80540ADF80C9008960995FFF772FC8C
:10A92000044620B9074A136843EA09031360204626
:10A9300014B0BDE8F0870E24F9E700BF622C0020B8
:10A9400060D90700B033002000B53B4B8BB01868CE
:10A95000019000F078FD002835D13848FFF762FCFF
:10A9600088BB374B3749502201A800F073FB08B170
:10A97000FEF743FA012103AA084600F0C3FB10BB0F
:10A98000172303A8ADF81C3000F0D0FBD8B92E482F
:10A9900000F092FBB8B99DF800300390012262F3F9
:10A9A0000303049062F3071301A88DF80030FFF74A
:10A9B00013FC40B99DF8053001A801338DF805302E
:10A9C000FFF708FC10B10BB05DF804FB07221F492C
:10A9D0006846FFF70DFC0028F5D10C23ADF80C30CC
:10A9E0001823ADF80E30ADF810004FF4C87303A86B
:10A9F000ADF81230FFF7FAFB0028E4D11448FFF756
:10AA0000F5FE0028DFD101461C2203A8FDF7A0FDBA
:10AA100040F6CD4304934FF48043059303238DF810
:10AA2000183003A80B4B099300F08EF80028CAD108
:10AA3000FFF7ACFCC7E700BF70D907000080070034
:10AA400061B107004C330020B9A4070074D9070096
:10AA50009C33002065A2070075DF704776DF7047E2
:10AA60007ADF70477BDF704737B5164B18884FF693
:10AA7000FF73984210D0144A144D1378297B013388
:10AA8000DBB2994213702C4608D31149FFF7E4FF5B
:10AA900010B1AB6903B1984703B030BD0023137008
:10AAA0002B7C33B13B21FFF7D9FF10B1AB6903B168
:10AAB00098476369002BEFD002A8002200F8042D0C
:10AAC000E9E700BFCA33002018340020CC3300204F
:10AAD0001034002037B5164B164A5B881188164C87
:10AAE000164D99420ED852889A420BD36369D3B15E
:10AAF00002A8012203E06369ABB102A8002200F8BA
:10AB0000042D0FE02A78002AF5D10D4861680078FD
:10AB1000A368002818BF19460A48FEF737FE10B18F
:10AB2000A36903B1984700232B7003B030BD00BF69
:10AB30000834002010340020CC330020C83300201B
:10AB400018340020E833002070B5054606460FCDC6
:10AB5000114C0FC495E80700104B84E80700002251
:10AB60001A7032680E489AB11368036053684360E4
:10AB7000FFF776FF78B90B4B0B484FF6FF721A8040
:10AB80000A4B0B4A00211970BDE87040FEF7ECBD7E
:10AB9000FFF768FFEEE770BDCC330020C83300201C
:10ABA00010340020CA3300207CD90700183400205C
:10ABB00069AA07000148FEF72FBE00BFE833002056
:10ABC00010B50388112B1BD002D8102B05D010BD57
:10ABD000122B39D0502B24D010BD1F4B82881A80E5
:10ABE00000F1100303CB1D4A1D4B10605160002281
:10ABF0001A701C4BDB8973BBBDE81040FFF76ABFBE
:10AC0000154B19484FF6FF721A80154B00221A7027
:10AC1000FEF702FEF8B1134B9B69E3B1BDE81040AB
:10AC20001847104CC288E3899A4214D1038A022B38
:10AC300011D1123000F01AF80028DDD10A48FEF7D1
:10AC4000EBFD40B1A369E8E700F1080303CB034A39
:10AC500010605160D0E710BDCA33002008340020D6
:10AC600018340020CC330020E8330020007800F0B6
:10AC700001007047BFF34F8F0549064BCA6802F4C5
:10AC8000E0621343CB60BFF34F8F00BFFDE700BF0F
:10AC900000ED00E00400FA05094B1B78062B0CD1EF
:10ACA000084B1B681A0708D1074B186800F0F00022
:10ACB000A0F130035842584170470020704700BF50
:10ACC000E00F00F0E40F00F0E80F00F00C4B1B78F1
:10ACD000062B10D10B4B1B681A070CD10A4B1868B6
:10ACE00000F0F003302B08D000F0E000A0F14003AA
:10ACF000584258417047002070470120704700BFFC
:10AD0000E00F00F0E40F00F0E80F00F008B5FFF7E7
:10AD1000C3FF10B1784B794A1A60FFF7D7FF28B10B
:10AD2000774B784A1B68C3F342331360FFF7B4FFD5
:10AD300020B1754AD36823F08073D360FFF7C6FF54
:10AD400040B14FF080430022C3F80C21C3F810211A
:10AD5000C3F83825FFF7A0FF10B16C4B03221A602F
:10AD6000FFF79AFF40B16A4B05221A6001229A67E9
:10AD700000229A603F225A60664B1B78062B09D14D
:10AD8000654B1B68190705D1644B1B6803F0F00382
:10AD9000502B68D0FFF79AFF28B1614B614A1B68BE
:10ADA00003F04F031360604AD2F8883043F4700315
:10ADB000C2F88830BFF34F8FBFF36F8F4FF010236F
:10ADC000D3F80C22D2071ED5584B0122C3F8042514
:10ADD000D3F80024002AFBD04FF01022D2F80C3216
:10ADE00023F00103C2F80C32504B1A46D3F800147A
:10ADF0000029FBD00021C3F80415D2F80034002B41
:10AE0000FBD0FFF737FFD3F80022002A03DBD3F88B
:10AE10000432002B23DA454B0122C3F80425D3F872
:10AE20000024002AFBD04FF010221521C2F8001296
:10AE3000D3F80024002AFBD04FF010231522C3F8CA
:10AE400004223A4B1A46D3F800140029FBD0002103
:10AE5000C3F80415D2F80034002BFBD0D1E7344BF3
:10AE6000344A1A6008BD4FF08052334BD2F80414B4
:10AE7000C3F82015D2F80814C3F82415D2F80C141E
:10AE8000C3F82815D2F81014C3F82C15D2F81414EE
:10AE9000C3F83015D2F81814C3F83415D2F81C14BE
:10AEA000C3F84015D2F82014C3F84415D2F824147E
:10AEB000C3F84815D2F82814C3F84C15D2F82C144E
:10AEC000C3F85015D2F83014C3F85415D2F834141E
:10AED000C3F86015D2F83814C3F86415D2F83C14DE
:10AEE000C3F86815D2F84014C3F86C15D2F844249E
:10AEF000C3F870254EE700BF74C007400DF0ADBA2F
:10AF0000440200103C050040F0ED00E0A0050040C8
:10AF100010560040E00F00F0E40F00F0E80F00F0E2
:10AF200058020010E40E004000ED00E000E0014097
:10AF3000642C00200090D00300C0004048DF704720
:10AF400010DF704760DF704761DF7047FDF752BF69
:10AF50000B4A92F81633C3F34113012B0CD9094B5A
:10AF6000986828B11A6842F480021A60002070477D
:10AF70004FF480031360704742F20200704700BF35
:10AF800000E100E0A43200202DE9F74F284B1B78A8
:10AF900003F0FF07002B43D0264D274E2B68346863
:10AFA000DFF89880DFF898A0DFF898B0B3FA83F361
:10AFB000B4FA84F45B096409C3B998F800307BBB28
:10AFC00001A8FFF7BBFF05282DD038B1FDF715FF0D
:10AFD00074B1B946002423464C46EDE72B6801982E
:10AFE0009847F5E7326818469047F4E7C4B91C461D
:10AFF00098F8003003F0FF0993B902A9BAF80030BD
:10B0000021F8043DDBF800301846FFF79DFF0528C6
:10B0100004D00028E6D0FDF7F0FEDCE7002CD8D005
:10B0200003B0BDE8F08F002CFAD13C46E0E700BF4A
:10B0300024340020283400201C3400202534002033
:10B040001A3400202C340020014B1878704700BFC0
:10B050002434002010B509B38C071FD1104C216097
:10B0600010490A80104A1360104A1368C3F3403332
:10B070001BB14FF40051C2F880100D49FFF760FF7B
:10B0800028B163B1094B4FF400521A6010BD094B4F
:10B0900001221A70BDE81040FFF75ABF072010BD0B
:10B0A0002C3400201A3400202034002000E100E07D
:10B0B0004DAF07002434002018B1034B1860002066
:10B0C00070470E20704700BF1C34002018B1034B9E
:10B0D0001860002070470E20704700BF2834002001
:10B0E00008B5074B1B682BB1984738B1BDE808403D
:10B0F000FDF783BEBDE80840FFF746BF08BD00BFAF
:10B100002034002070B5144605460E461C2200214E
:10B110002046FDF71DFA01234FF00002238022751F
:10B120002672657205B1A372002070BD07B5064B8B
:10B13000019302A9019B41F8083DFFF703FF019B22
:10B1400003B05DF804FB00BF002C002008B511B16E
:10B150000020FDF752FEBDE80840FFF715BF0000D4
:10B160000021024A0846FDF75DBF00BF4DB1070050
:10B1700008B500F039F808BD13DF7047F0B5034695
:10B18000186880F308885868FF2464B2EFF30585D7
:10B19000002D01D1A64600472546064621273FBA85
:10B1A000F0B40024002500260027F0B4F92040B2B6
:10B1B000004700BFF0BD00BF10B5044600F043F9E2
:10B1C00068B9074B4FF0FF32C3F880202046FFF7E5
:10B1D000D3FF20B92046BDE81040FFF7CFBF10BD18
:10B1E00000E100E0FDF77EBF13B502AC002344F898
:10B1F000043D00F0EDF9204600F0A6FA08B1012365
:10B200000193FDF739FE08B101230193019CCCB1F4
:10B21000144B154A05210020FEF762FA08B1FDF72C
:10B22000ECFD124A14210820FDF7D8FE08B1FDF705
:10B23000E4FD00F0F9F9044680B9FDF7E7F9FDF700
:10B2400051FFFCE700F02AFB0028E1D000F026FBCC
:10B2500020B143F208031868FFF7AEFF204602B0A2
:10B2600010BD00BF51980700803500203034002009
:10B2700010B40A4A136823F0010439B923F0030318
:10B280001360436833B15DF8044B184744F002047F
:10B290001460F6E75DF8044B704700BFF8350020F6
:10B2A00008B568B1FEF704FC08B1082008BD0648DF
:10B2B000FFF70CFF0028F8D1044B04221A6008BDE8
:10B2C000024B186008BD00BFDD9B0700F835002069
:10B2D0002DE9F041DFF884801C46D8F8003013F0E7
:10B2E000040F86B006460D46174616D09A0729D495
:10B2F00043F00103C8F800300A4600940146BBB28F
:10B300001548FEF7DFFB28B9D8F8003043F00103F9
:10B31000C8F8003006B0BDE8F081A9B1A0B105437E
:10B3200015F0030512D19AB1FEF732FF94B102A8CD
:10B3300029468DF8085003940496ADF81470A04780
:10B340002846E7E70A20E5E70320E3E70620E1E7F0
:10B350000420DFE72046DDE7742C0020F8350020CC
:10B360002DE9F043234E33680F46590785B0054653
:10B37000144615D59A0737D443F0010333600146CC
:10B380002346BAB21C48FEF7E5FB336828B123F028
:10B390000103336005B0BDE8F08343F00103F8E733
:10B3A000C0F30B0313BBC0F30F393E468046404643
:10B3B000FEF7D4FE013E08F58058F8D105EB0735BD
:10B3C000B4B1102231466846FDF7C2F82D0B0123B7
:10B3D000684631468DF800300194ADF80890ADF81C
:10B3E0000A50A0473046D5E70A20D3E70620D1E728
:10B3F0002046CFE7F8350020742C002018DF704776
:10B4000030B585B0054610220C4668460021FDF790
:10B410009FF8A408684601950294FFF7EFFF05B076
:10B4200030BD1FB59208C2F3090353B9012302903E
:10B430006846009301910392FFF7E0FF05B05DF8C5
:10B4400004FB0920FAE71FB5102200216846FDF72A
:10B450007FF8022368460093FFF7D0FF05B05DF840
:10B4600004FB1FB5032301909208684600930291E4
:10B470000392FFF7C3FF05B05DF804FB09B9034B66
:10B480001970034B1B6803B118477047FC35002047
:10B4900000360020204B21491A68214B00BF00BF15
:10B4A00000BF00BF00BF00BF00BF00BF8A422FD057
:10B4B00000BF00BF00BF00BF00BF00BF00BF00BF94
:10B4C00000BF00BF00BF00BF00BF00BF00BF00BF84
:10B4D00000BF00BF00BF00BF00BF00BF00BF00BF74
:10B4E00000BF00BF00BF00BF00BF00BF00BF00BF64
:10B4F00000BF00BF00BF00BF00BF00BF00BF00BF54
:10B5000000BF00BF00BF00BF00BF00BF00BF00BF43
:10B51000013BC3D1704700BF642C00200024F4001D
:10B52000A086010008B5FEF7B5FB00B908BDFFF71E
:10B53000B1FFFDF7D7FDF6E7002258210148FEF7DD
:10B54000CFB900BF08360020F8B51B4C064625468B
:10B55000237893B901232370184B194C1E60FFF711
:10B56000E1FF002201212046FFF7FAFE0728F6D06E
:10B5700040B100232B700320F8BDFFF78BFFFDF7D0
:10B58000B1FDE5E7FFF7D8FF0E490F4F08604FF414
:10B59000AE720E480D4E0A4C01F0F5FFFFF7C2FFE8
:10B5A0003B46572231462046FFF792FE0728F5D04A
:10B5B0000028DED1F8BD00BFFC3500200036002099
:10B5C00000F00700043600207DB40700603700203B
:10B5D00010B5124B124C134900221A7020464FF43A
:10B5E000AE7201F0D0FF226801320FD14FF4AE727B
:10B5F00000210B48FCF7ACFF012300206360FFF73C
:10B60000A3FF48B1BDE81040FDF7F7BBFFF794FF7B
:10B6100023689842EAD110BD10BD00BFFC35002060
:10B620000436002000F0070070B5084E084CA41B3B
:10B63000E4080025A54201D1002070BD56F8353040
:10B6400098470028F9D10135F4E700BF842C002089
:10B650008C2C002070B5084E084CA41BE408002573
:10B66000A54201D1002070BD06EBC5035B68984779
:10B670000028F8D10135F3E7842C00208C2C002021
:10B68000044A0023036043608360136353631361C0
:10B6900053617047043600202DE9F041184E1949D6
:10B6A000726B336B02F6FF74E41A0C40A50805F6C2
:10B6B000FF7503F580570D4003EB00080AB1934274
:10B6C0001BD02A4641463846FFF7ABFEB0B92A46A2
:10B6D00041463846FFF7C5FE80B9A542736B8CBF63
:10B6E0000446641B1B1B00202F44A8443363FFF750
:10B6F0002BFF002CE5D1BDE8F0810020BDE8F081F2
:10B700000436002000F0FFFF70B50D4B0D685C6B38
:10B710002D1B04440E462A4621460A48FFF7A1FE87
:10B72000014638B93046FFF7ABFFBDE87040084628
:10B73000FFF70ABF29462046BDE87040FFF760BE0C
:10B7400004360020008007002DE9F04743F208038B
:10B7500080461E684F4B1A69012A994614D05B69CE
:10B7600093B1D9F8184004F6FF7424F47F6424F0F0
:10B770000F04344409F12407BB68A52B71D007D806
:10B78000012B14D000257BE0344609F11807F3E7BC
:10B79000AA2B78D0AC2BF5D12046FFF77DFF0546CC
:10B7A00000286AD139462046FFF7AEFF64E0D9F899
:10B7B0001430012BE6D1D9F83070D9F824A03E44DA
:10B7C000AAEB0707B7F5805F4FF000024FF00101C9
:10B7D0003046B84628BF4FF48058FFF7C1FD0546F4
:10B7E00000284DD10346424621463046FFF770FD02
:10B7F0000546002844D1424621463046FFF731FE37
:10B80000054600283CD1024601212046FFF7A8FD4D
:10B810000546A8BBD9F830304344C9F83030FFF7AB
:10B8200093FEB7EB080746444444CBD143F20803E8
:10B830003A4651461868FEF753F8D9F8283098422E
:10B8400004BFC9F81C000123134804BFC9F8203005
:10B85000C9F818A0FFF714FF0020BDE8F047FFF774
:10B8600073BE2046FFF718FF054630B93846FFF78C
:10B8700007FF2846FFF768FE05460123C8F8003099
:10B880002846BDE8F08739462046BDE8F047FFF777
:10B890003BBF00BF043600202836002010B50B4CFB
:10B8A000236A012B0DD8E3696BB143F20803002230
:10B8B000A1691868FEF714F8E3691B1A5842584149
:10B8C00010BD002010BD012010BD00BF04360020B7
:10B8D00070B5194C43F2080325681B68A5F540555F
:10B8E000ED1A854201D2042070BD1360134B1E6A0D
:10B8F000012E1CD19C6904F6FF7424F47F6424F0AB
:10B900000F042D1BA84205D90029ECD11E615961F5
:10B91000183306E0002119615E6111680C4414605F
:10B920002433002218605A609A60104670BD0022CD
:10B930001A615A61ECE700BF1410001004360020B1
:10B940000023C2600160416083608B781A44026109
:10B9500091F903301A4442610878003018BF012081
:10B96000704710B542681178034600293AD002F1B9
:10B970000C014160147B2CB9C2680168FFF7E0FF3D
:10B98000204610BD5078117900F03004302C1BD1C6
:10B99000547B04F03004302C16D190781969091AC0
:10B9A00019610021507810F0300F02BF9868013003
:10B9B0009860907B084419690144196192F90F203D
:10B9C00011445961012010BD00F0F004202C03D176
:10B9D000507910FB01F1E5E700F0C000802808BFB6
:10B9E0000421DFE7084610BD70B5456804460E46E1
:10B9F00063681A78B24204D15B7803F00F03082B16
:10BA000007D12046FFF7ADFF63689D42F0D10020CB
:10BA100070BD012070BD43681A44426011B1013904
:10BA2000934201D10120704713F8010B01F8010F77
:10BA3000F6E770B543685B7803F00F02082A86B01A
:10BA40001FD103691C6800260CB906B070BD2368BD
:10BA500026739D68626829466846FFF771FF636830
:10BA6000049304F10C0305936B7803F0C003802B5F
:10BA700008BF231D684608BF0493FFF7DAFFA468D8
:10BA8000E2E713F0C0021FD103F0300110290CD1FE
:10BA900043691A7043685A7802F00F02072A09D1E5
:10BAA0000169986800F018F8CFE79906F2D5436964
:10BAB0001A70CAE7996800691A7911B101F063FD3B
:10BAC000C3E7FCF745FDC0E7802ABED1016900222B
:10BAD0009B060A60B9D5EAE77FB50A460146684683
:10BAE000FFF72EFF30B16846FFF7A3FF6846FFF768
:10BAF00038FFF7E707B05DF804FB2DE9F3418368F1
:10BB00000446884623B90027384602B0BDE8F081D4
:10BB1000036801220DF10701984707460028F2D07B
:10BB2000A3689DF80750013B2A06A3601AD505F0CB
:10BB30007F050726A368002BE5D0236801220DF1BD
:10BB40000701204698470028DDD0A3689DF807200C
:10BB5000013BA36002F07F03B3401D43130606F1CF
:10BB6000070602D4C8F80050CEE7232EE2D1CAE778
:10BB700030B5044685B01546A9B90268114B9A4202
:10BB800011D0102D06D82A4669462046FFF7F0FF4F
:10BB900005B030BD102269462046FFF7E9FF0028B6
:10BBA000F6D0103DEDE7A3689D4201D90020EFE7F4
:10BBB00023682A46204698470028F7D0A3685D1BD3
:10BBC000A560E5E717BA070073B50D4601A906465B
:10BBD0001446FFF792FF88B1019A511C10D26B787E
:10BBE00003F0C003802B0BD02B79994208D8214653
:10BBF0003046FFF7BDFF019B0022E25402B070BD4A
:10BC00000020FBE773B50D4601A906461446FFF771
:10BC100074FF90B1019AFF2A11D8511C0FD26B7892
:10BC200003F0C003802B0AD02B79994207D8214614
:10BC3000304601F8012BFFF79BFF02B070BD0020DA
:10BC4000FBE7000010B58260024C046000224160F6
:10BC5000C26010BD17BA07002DE9F34704460F462E
:10BC60004FF000084FF000090025A36803B32368D4
:10BC700001220DF10701204698470646C0B1A3688E
:10BC80009DF807A0013B2A46A3600AF07F0000212F
:10BC900001F05EFC1AF0800F48EA000849EA010949
:10BCA00005F1070502D1C7E9008902E0462DDCD184
:10BCB0000026304602B0BDE8F08737B50D4669462C
:10BCC0001446FFF7C9FF68B12B79082B0CD1DDE9C9
:10BCD0000001C4E90001DDE900238B4206BF824276
:10BCE0000120002003B030BD042B04D1DDE90001A8
:10BCF00020600021EFE7022B03D10098208080B262
:10BD0000F7E7012B05D1DDE90001207000F0FF000D
:10BD1000EFE70020E6E737B50D4669461446FFF722
:10BD20009BFF30B12A79082A05D1DDE90023C4E957
:10BD3000002303B030BD009B042A18464FEAE3718C
:10BD400008D123601A460B468B4206BF824201206F
:10BD50000020EEE7022A04D11BB223801AB2D317C7
:10BD6000F2E7012A03D15BB223705AB2F7E7002051
:10BD7000DFE7F7B50C46002119702170116001A9A9
:10BD8000074615461E46FFF7B8FE30B9BB6813B923
:10BD900001233370002003B0F0BD01990029F7D0D2
:10BDA000CB0801F007012B602170F4E713B50446BE
:10BDB00005291FD8DFE801F0030F151E1E1C012204
:10BDC00001A92046FFF7D4FE18B19DF90430002BDD
:10BDD000F5DB02B010BD082200212046FFF7C8FEA7
:10BDE000F7E701A9FFF789FE0028F2D0019AF3E7EF
:10BDF0000422F1E70020ECE773B50D4601A90446E3
:10BE0000FFF77BFE064618B90026304602B070BD2B
:10BE100094E80F0085E80F0001998A42F4D3A960E5
:10BE2000A3685B1AA360F0E72DE9F04355686B78CF
:10BE300013F0C00C89B006468E46144604D0BCF1FF
:10BE4000400F6AD0002546E003F00F025D4903F081
:10BE50003003102B51F822701DD006D8002BF1D1E1
:10BE600022692946B847054635E0202B19D0302BEA
:10BE7000E8D1636929781970072A0AD163682069B3
:10BE80001A796146FCF764FB636821699868FFF7DB
:10BE900023FE22693EE0636901221A70226961680B
:10BEA000E0E7BEF1020FD4F8148027D1042A25D888
:10BEB00004A9FFF7A1FF05460028C3D0069B2BB1BC
:10BEC000616898F800304A799A4208D8059B7360F7
:10BED000069B002BB6D1284609B0BDE8F08308794F
:10BEE000226900FB032204A8B84728B198F8003063
:10BEF000013388F80030E1E70546E7E798F80030BD
:10BF00006A799A429ED922692979581C88F80000DA
:10BF100001FB032261683046A4E717693B6807F11B
:10BF2000040913B9FFF742FF9DE7022913D104A9C1
:10BF3000FFF762FF002885D03B6861684A4604A885
:10BF40009847054600283FF47DAF069B002BF3D1B0
:10BF5000059B7360BFE701292AD009D305297FF427
:10BF600071AF04220DEB0201FFF702FE042524E06D
:10BF700000250DF1040801350B2D3FF463AF0122BC
:10BF800041463046FFF7F4FD00283FF45BAF18F957
:10BF9000013B002BEFDB0C4B049301AB059300231B
:10BFA000069507933B6861684A4604A898475AE794
:10BFB000082201A9FFF7DCFD082500283FF442AF65
:10BFC000E9E700BF80D9070017BA07002DE9F04F55
:10BFD00091B00026044604A802960396FFF7B0FC31
:10BFE000A3683BBB059B069C5D7804A8FFF7B9FCE2
:10BFF0000028F7D115F0300F03D1059B1B7803B152
:10C000000134002C00F0B4806209002302A993429D
:10C0100040F0A78010AA02EB830304F01F04C4F1D0
:10C0200020044FF0FF3053F8383CE040C31A584228
:10C0300058410EE00DF1030301AA0DF10201204663
:10C04000FFF797FE814638B99DF80330002BC9D120
:10C05000002011B0BDE8F08F019904A8FFF7C4FCDF
:10C0600000285AD1019B9E421DD8059D059A537800
:10C0700003F00F03082B7DD004A8FFF772FC059B8B
:10C080009D42F3D14FF0FF36019FBE420BD8089B73
:10C09000D4F808809DF802A01D68A3680DB19845EA
:10C0A00009D098459CD19DF802102046FFF77EFEEE
:10C0B000002895D1CCE72B68D3F800B0BBF1000F76
:10C0C00008D053463A4629462046D8470028BFD0D4
:10C0D000AD68E2E7D3F808B09BF800309F421AD170
:10C0E0006A6859460AA8FFF72BFC6B680E9305F1A6
:10C0F0000C030F939BF8013003F0C003802B04BFA7
:10C100002B1D0E934FF001032B730AAA51462046B4
:10C11000FFF78AFEDAE74846D8E7059B5B7813F01D
:10C12000300F0FD1069A3F2A0CD8510910AB03EB00
:10C13000810102F01F020123934051F8382C134370
:10C1400041F8383CE5682DB104AB9DF80220019917
:10C150002046A84704AA9DF802102046FFF764FE77
:10C16000A6E751F8235001357FF473AF01334EE752
:10C1700001206EE7167887E770B50C46064615462F
:10C1800011462046FFF7A8FC2A4621463046BDE866
:10C190007040FFF71BBFF0B585B00C468D6869464F
:10C1A00007461646FFF728FE68B1A06858B16378C5
:10C1B00003F03003202B32462946684605D1FFF7AD
:10C1C000DBFF019B7B6005B0F0BDFFF7FFFEF8E7EA
:10C1D000D3B50C466946FFF73FFD70B1DDE900239A
:10C1E000002702F001065B084FEA320256EA070117
:10C1F0001CBFD243DB43C4E9002302B0D0BD37B536
:10C200000D4669461446FFF7E3FF68B12B79082B0A
:10C210000CD1DDE90001C4E90001DDE900238B4216
:10C2200006BF82420120002003B030BD042B03D1A1
:10C2300000982060C117F0E7022B04D1BDF900007F
:10C24000208000B2F6E7012B04D19DF90000207098
:10C2500040B2EFE70020E7E713B504220C460DEBF0
:10C260000201FFF785FC08B1019B236002B010BDFD
:10C270001146FFF7F1BF13B508220C466946FFF7D8
:10C2800077FC18B1DDE90023C4E9002302B010BD3A
:10C290001146FFF7F0BF8B1802448B4200D1704764
:10C2A00013F8010D02F8010DF7E710B5013A52B28B
:10C2B000002A01DA002010BD13B250F8234051F8D3
:10C2C00023309C4203D8F1D24FF0FF3010BD012043
:10C2D00010BD000000000000000000000000000091
:10C2E000C3F10803DB0070B50133002403A500BFD0
:10C2F0005B1920C940CAAD1920C0184720C940CADF
:10C30000754120C020C940CA754120C020C940CA1B
:10C31000754120C020C940CA754120C020C940CA0B
:10C32000754120C020C940CA754120C020C940CAFB
:10C33000754120C06441204670BD00BF0000000070
:10C34000C3F10803DB0070B50133002403A500BF6F
:10C350005B1920C940CAAD1B20C0184720C940CA7C
:10C36000B54120C020C940CAB54120C020C940CA3B
:10C37000B54120C020C940CAB54120C020C940CA2B
:10C38000B54120C020C940CAB54120C020C940CA1B
:10C39000B54120C06441B4FA84F0400970BD00BFCB
:10C3A0002DE9F04F08B4F8CA04B451F8042BA3FBEC
:10C3B000028940F8048B4FF0000AE4FB629A4FF0C8
:10C3C000000BE5FB62AB4FF0000CE6FB62BC4FF0EC
:10C3D000000EE7FB62CE51F8042B4FF00008E3FBA0
:10C3E000628940F8048BE4FB629AE5FB62ABE6FBF2
:10C3F00062BCE7FB62CE51F8042B4FF00008E3FB70
:10C40000628940F8048BE4FB629AE5FB62ABE6FBD1
:10C4100062BCE7FB62CE51F8042B4FF00008E3FB4F
:10C42000628940F8048BE4FB629AE5FB62ABE6FBB1
:10C4300062BCE7FB62CE51F8042B4FF00008E3FB2F
:10C44000628940F8048BE4FB629AE5FB62ABE6FB91
:10C4500062BCE7FB62CE40F8049B40F804AB40F8B6
:10C4600004BB40F804CB40F804EB0CBC052B00F0F7
:10C470001E810C68A0F11400A1F11401A2F11402B4
:10C4800052F804EB4FF0000550F8046BE4FB6E56D5
:10C4900052F804EB50F8047BE4FB6E6752F804EBAF
:10C4A00050F8048BE4FB6E7852F804EB50F8049BD0
:10C4B000E4FB6E8952F804EB50F804ABE4FB6E9A8F
:10C4C000A0F1140052F8044B51F804EB4FF0000CAB
:10C4D000E4FB6EC540F804CB51F804EBE4FB6E5668
:10C4E00040F8045B51F804EBE4FB6E6740F8046B22
:10C4F00051F804EBE4FB6E7840F8047B51F804EB50
:10C50000E4FB6E8940F8048B51F804EBE4FB6E9A6F
:10C51000A0E80006062B00F0CA800C68A0F1180005
:10C52000A1F11801A2F1180252F804EB4FF0000536
:10C5300050F8046BE4FB6E5652F804EB50F8047BA1
:10C54000E4FB6E6752F804EB50F8048BE4FB6E7862
:10C5500052F804EB50F8049BE4FB6E8952F804EBAC
:10C5600050F804ABE4FB6E9A52F804EB50F804BBAD
:10C57000E4FB6EABA0F1180052F8044B51F804EB49
:10C580004FF0000CE4FB6EC540F804CB51F804EB0F
:10C59000E4FB6E5640F8045B51F804EBE4FB6E6775
:10C5A00040F8046B51F804EBE4FB6E7840F8047B30
:10C5B00051F804EBE4FB6E8940F8048B51F804EB6E
:10C5C000E4FB6E9A40F8049B51F804EBE4FB6EAB7D
:10C5D000A0E8000C072B6AD008B40C68A0F11C007E
:10C5E000A1F11C01A2F11C0252F804EB4FF000056E
:10C5F00050F8046BE4FB6E5652F804EB50F8047BE1
:10C60000E4FB6E6752F804EB50F8048BE4FB6E78A1
:10C6100052F804EB50F8049BE4FB6E8952F804EBEB
:10C6200050F804ABE4FB6E9A52F804EB50F804BBEC
:10C63000E4FB6EAB52F804EB50F804CBE4FB6EBCA9
:10C64000A0F11C0052F8044B51F804EB4FF000032A
:10C65000E4FB6E3540F8043B51F804EBE4FB6E5606
:10C6600040F8045B51F804EBE4FB6E6740F8046BA0
:10C6700051F804EBE4FB6E7840F8047B51F804EBCE
:10C68000E4FB6E8940F8048B51F804EBE4FB6E9AEE
:10C6900040F8049B51F804EBE4FB6EAB40F804ABAC
:10C6A00051F804EBE4FB6EBCA0E8001808BCBDE840
:10C6B000F08F2DE9F04FB1E8005E06B4AAFB091235
:10C6C0004FF00003EBFB69234FF00004ECFB6934EF
:10C6D0004FF00005EEFB69454FF00006EBFB6A6387
:10C6E000ECFB6A344918524176415B41A9FB097859
:10C6F0004FF0000949F1000918EB0108A0E880019A
:10C70000AAFB0A78574158EB0608A0E88001EEFB27
:10C710006A454FF0000A4AF1000A4FF00001ECFBB5
:10C720006B14EEFB6B454FF00002EEFB6C255FEAED
:10C7300059094941644152416D4149F10009EBFBFE
:10C740006B3A1AEB010AA0E80804ACFB0C6A6641DC
:10C750005AEB020AA0E84004AEFB0E6A6E415AEBA7
:10C76000090AA0E8400406BC052A00F0E680A0F112
:10C770001400A1F11401B1E8E043A5FB0E344FF021
:10C780000005E6FB6E454FF00006E7FB6E564FF0E6
:10C790000007E8FB6E674FF00008E9FB6E784FF08A
:10C7A0000009DB1864416D4176417F4158EB080870
:10C7B00059F1000950F804CB13EB0C0350F804CBEB
:10C7C00054EB0C0450F804CB55EB0C0550F804CB9B
:10C7D00056EB0C0650F804CB57EB0C0758F1000849
:10C7E00059F10009A0F11400EEFB0E89A0E8F8034E
:10C7F000062A00F0A280A0F11800A1F11801B1E80A
:10C80000E047A5FB0E344FF00005E6FB6E454FF008
:10C810000006E7FB6E564FF00007E8FB6E674FF02F
:10C820000008E9FB6E784FF00009EAFB6E894FF0D3
:10C83000000ADB1864416D4176417F4158EB0808DE
:10C8400059EB09095AF1000A50F804CB13EB0C0319
:10C8500050F804CB54EB0C0450F804CB55EB0C050A
:10C8600050F804CB56EB0C0650F804CB57EB0C07F2
:10C8700050F804CB58EB0C0859F100095AF1000AA2
:10C88000A0F11800EEFB0E9AA0E8F807072A54D092
:10C89000A0F11C00A1F11C01B1E8E04FA5FB0E3492
:10C8A0004FF00005E6FB6E454FF00006E7FB6E56C5
:10C8B0004FF00007E8FB6E674FF00008E9FB6E7869
:10C8C0004FF00009EAFB6E894FF0000AEBFB6E9A0D
:10C8D0004FF0000BDB1864416D4176417F4158EB0E
:10C8E000080859EB09095AEB0A0A5BF1000B50F8EA
:10C8F00004CB13EB0C0350F804CB54EB0C0450F8AE
:10C9000004CB55EB0C0550F804CB56EB0C0650F855
:10C9100004CB57EB0C0750F804CB58EB0C0850F83D
:10C9200004CB59EB0C095AF1000A5BF1000BA0F1A2
:10C930001C00EEFB0EABA0E8F80FBDE8F08F002363
:10C9400010B51C465AB2914200DC10BD40F823409D
:10C950000133F7E72DE9F047B3F9024088461E4658
:10C9600004F11F012023073491FBF3F708234FFA4A
:10C9700087F994FBF3F4944228BF144649460546D0
:10C98000FFF7DDFF22464146FFF785FCB6F902308E
:10C99000E4009C4221D9E41A05EB87010022C4F18E
:10C9A00020078D420FD324364A4629463046FFF7EA
:10C9B0007CFC012811D04B46324629462846BDE86A
:10C9C000F047FFF7BDBC51F8040C20FA04F3134301
:10C9D00041F8043D00FA07F2E3E7BDE8F08710B53F
:10C9E00000231A465CB2A14203DCB2FA82F040098D
:10C9F00010BD50F8234001332243F3E74A110123CD
:10CA000050F8220001F01F0103FA01F108407047BD
:10CA1000013949B2002904DA013149B231B9084675
:10CA2000704750F82130002BF2D0F5E701F1804338
:10CA3000013B50F82330002023B9013900EB4111AC
:10CA400008B270475B080130F6E710B500235CB20E
:10CA5000A24200DC10BD51F8234040F823400133CE
:10CA6000F5E70000F0B5082289B00C460646FFF74E
:10CA7000ECFFCB6A03930B6B04934B6B05938B6BAF
:10CA80000693CB6B0793002708236A4669466846DE
:10CA9000029701970097FFF723FC082305466A4693
:10CAA00031463046FFF71CFC236B0393636B049302
:10CAB000A36B0593E36B0693054408236A46694616
:10CAC00068460797FFF70CFC082305446A46314681
:10CAD0003046FFF705FC236A0093636A0193A36A5B
:10CAE0000293A36B0693E36B0793054408236A46FE
:10CAF00031463046059704970397FFF7F1FB636AC9
:10CB00000093A36A0193E36AA26B0293636B03939E
:10CB100004920693E26B236A0592054407936A46E2
:10CB2000082331463046FFF7DBFBE36A0093236BB3
:10CB30000193636B0293236A0693A36A07930544E8
:10CB400008236A4631463046059704970397FFF756
:10CB5000F7FB236B0093636B0193A36B0293E36B6F
:10CB60000393636A0693E36A07932D1A08236A46C0
:10CB70003146304605970497FFF7E2FB636B00935D
:10CB8000A36B0193E36B0293236A0393636A049399
:10CB9000A36A0593236B07932D1A08236A4631462F
:10CBA00030460697FFF7CCFBA36B0093E36B019332
:10CBB000636A0393A36A0493E36A0593636B079321
:10CBC0002D1A08236A463146304602970697FFF72A
:10CBD000B7FB2D1A0D4C0FD435B90822314620462B
:10CBE000FFF763FB01280FD0082322463146304669
:10CBF000FFF7A6FB2D1AEFE7082322463146304601
:10CC0000FFF76EFB2D18F7D409B0F0BDA8D90700C7
:10CC100030B5013A52B20023002A03DAB3FA83F0A6
:10CC2000400930BD15B2013A50F8254051F8255061
:10CC30006C40234352B2EFE700EB810100238842AE
:10CC400000D3704751F8042C43EA520341F8043DE5
:10CC5000D307F4E770B5036813F0010506461446E0
:10CC600005D013460A460146FFF73AFB0546214622
:10CC70003046FFF7E1FF45B104F18042013A56F832
:10CC8000223043F0004346F8223070BD70B59DF964
:10CC900010401E4623460546FFF722FB30B92246C8
:10CCA00029463046FFF701FB012807D023463246CC
:10CCB00029462846BDE87040FFF742BB70BD70B5FD
:10CCC0009DF910401E4623460546FFF739FB38B153
:10CCD0002346324629462846BDE87040FFF700BB90
:10CCE00070BD2DE9F04FA5B01D46039114AB294648
:10CCF0008046104617460293FFF78AFEC0EB851068
:10CD000004B2634203F01F034FF0200694FBF6F6D3
:10CD100076B204F01F0904A858BFC3F100093146D8
:10CD2000FFF70DFEB9F1000F30B22BDD04AB00228E
:10CD300003EB8000C9F1200E1346AB4217D32FB28C
:10CD40007B00019304AB03EB870705F1FF3924ABAC
:10CD5000012603EB8909002C55DB24AB0022C6F128
:10CD60000100964603EB860A03EB80002DE057F89E
:10CD7000236006FA09F10A4340F8232026FA0EF24E
:10CD80000133DAE704AB2A46394603EB8000FFF7AC
:10CD90005CFED4E70FFA81FC5AF8883C53F82CB0BB
:10CDA00024AB03EB810151F8803CABEB0303A3EB15
:10CDB0000E039B4504D034BF4FF0010E4FF0000E20
:10CDC00050F8881C41F82C300132019B51B2994235
:10CDD000E0DBA6EB0E035E42294604A85E41FFF7A6
:10CDE0002BFF24AB03EB8503294653F8802C59F81D
:10CDF000803C384643EAC273013C49F8803C24B287
:10CE0000FFF71AFFA7E724AB03EB86062A4656F87E
:10CE1000881C4046FFF719FE25B0BDE8F08F70B5BD
:10CE200090B005469DF950401E4668462346FFF7E0
:10CE3000B7FA2346324669462846FFF752FF10B03C
:10CE400070BD30B51C4691B0054693F90030684678
:10CE5000FFF7A6FAD4F8AC3069462846984711B0D7
:10CE600030BD30B5144691B0054692F900206846B1
:10CE7000FFF71FFCD4F8AC3069462846984711B03C
:10CE800030BD2DE9F04115468AB00446884620227F
:10CE9000002102A8FBF75CFB2E1D95F9007003230F
:10CEA0002A46414620460293FFF7DBFF334602AA9B
:10CEB000214620460097FFF702FF2B4642462146B7
:10CEC0002046FFF7BEFF0097334605F18402214656
:10CED0002046FFF7DBFE0AB0BDE8F0812DE9F04700
:10CEE00093F9006092B004468946104631461546D3
:10CEF0009846FFF774FD002840F09380424649466B
:10CF000002A8FFF7AEFF434602AA21460AA8FFF790
:10CF100098FF02A908464246FFF7A3FF43462A4668
:10CF200049464846FFF78DFF08F104074246294667
:10CF30002846FFF796FF3B462A46214620460096A4
:10CF4000FFF7A4FE3B462A46294628460096FFF7EF
:10CF50009DFE3B462A46214628460096FFF7AFFE37
:10CF600043462A4621462046FFF76BFF3B462246B2
:10CF7000214628460096FFF789FE3B4600962A4642
:10CF800021462046FFF782FE2368DB074CD5334657
:10CF90003A4621462046FFF7A3F93146824620460D
:10CFA000FFF74AFE06F18043013B54F8230040EAB4
:10CFB000CA7044F82300424621462846FFF751FF35
:10CFC0003B460AAA294628460096FFF778FE3B46CC
:10CFD0000AAA294628460096FFF771FE0AA90846C4
:10CFE0003B462A460096FFF76AFE43460AAA2146B8
:10CFF0002046FFF726FF02AA3B4610462146009630
:10D00000FFF75DFE324629462046FFF71EFD3246F9
:10D0100049462846FFF719FD324602A94846FFF760
:10D0200014FD12B0BDE8F08731462046FFF704FE3C
:10D03000C1E72DE9F0438BB01446129D15F9046B3E
:10D0400000961F46804689462B460246214602A886
:10D05000FFF735FE02A9129A0846FFF702FF129B5E
:10D0600002AA41464046FFF7ECFE129B02AA214667
:10D070002046FFF7E6FE2B464A46394638460096DC
:10D08000FFF71DFE129A394602A8FFF7EAFE02A931
:10D090002B46424608460096FFF711FE02A92B4692
:10D0A000224608460096FFF70AFE2B4642462146D6
:10D0B00020460096FFF703FE129B2246494648464B
:10D0C000FFF7BFFE2B4602AA414620460096FFF717
:10D0D000F6FD129B224639463846FFF7B2FE2B4634
:10D0E0004A46394638460096FFF7E9FD324602A91E
:10D0F0002046FFF7AAFC0BB0BDE8F083F0B515465B
:10D1000089B01C4607460E461A4629466846FFF770
:10D11000A8FE23466A4639463846FFF792FE234664
:10D120002A4669466846FFF78CFE23466A46314622
:10D130003046FFF786FE09B0F0BDF0B50F46A1B04E
:10D1400006461946384615461C46FFF748FC28B1E6
:10D1500021463046FFF7F3FB21B0F0BD22463946A9
:10D160006846FFF772FC2246294608A8FFF76DFCC7
:10D17000214610A8FFF7E3FB0123214618A81093CE
:10D18000FFF7DDFB224608A96846FFF78EF828B9AD
:10D19000224610A93046FFF758FCDDE7009BDA076E
:10D1A00009D421466846FFF747FD2246294610A8C4
:10D1B000FFF750FDE6E7089BDB0707D4214608A8E8
:10D1C000FFF73AFD2246294618A8F1E70028234632
:10D1D0001CDD08AA69466846FFF7B2F82146684692
:10D1E000FFF72AFD224618A910A8FFF75EF80028CD
:10D1F00005DA10A923462A460846FFF771F810A958
:10D20000234618AA0846FFF79BF8CEE708A96A4606
:10D210000846FFF795F8214608A8FFF70DFD2246BE
:10D2200010A918A8FFF741F8002805DA18A9234625
:10D230002A460846FFF754F818A9234610AA0846BC
:10D24000FFF77EF8BEE7000000487047A4D907004A
:10D250002DE9F04FEDB01F46DDF8D8810590B8F903
:10D26000026098F9005020231F3696FBF3F676B241
:10D2700006F1FF3924AB002443F829406CAB03EBE3
:10D2800089034CA88A469346394698F9012043F809
:10D29000804C43F8604CFEF7FEFF98F9012054A83B
:10D2A000B918FEF7F8FF29464CA8FFF798FB074688
:10D2B000002840F02981294654A8FFF790FB0390ED
:10D2C000002840F0238108F1240332464CA9184677
:10D2D0000293FEF7EAFF012840F01A81324654A972
:10D2E0000298FEF7E2FF0128069040F011811CAC85
:10D2F0000CAF3346029A54A92046FFF71EFF039B4A
:10D3000047F829305A46514638464346FFF722FB34
:10D3100039463846029B00962246FFF780FD0DF500
:10D32000B879029B009622464CA914A8FFF777FD16
:10D3300048462A460599FFF788FBAB0009EB030A2C
:10D340000793059BA900591808F1440B50462A463B
:10D35000FFF77BFB59462A4634A8FFF776FBAB0064
:10D360000BEB03012A463CA8FFF76FFB08F104030F
:10D37000494634AA204600950493FFF7A0FC534683
:10D380004A463CA934A8CDF80080FFF752FE2B4650
:10D39000049A21462046FFF7D0FE224651464846D1
:10D3A0004346FFF7ABFE039B08933146059B0A9368
:10D3B0003846CDF824B0CDF82C90FFF729FB314644
:10D3C000814614A8FFF724FB8145B8BF81461FFAA8
:10D3D00089F909F1FF3B0FFA8BFB59463846FFF7F5
:10D3E0000DFB5946071C14A818BF0127FFF706FBC1
:10D3F000002814BF022300231F430DF1200A2A46F0
:10D400005AF8277024A83946FFF71FFB0DF1B00B1F
:10D41000AB00F9182A465846FFF717FB2946204665
:10D42000FFF78DFAA9F10209069B23600FFA89F92B
:10D430000DF1900AB9F1000F20DA2B46049A21462B
:10D440002046FFF77AFE4346224659465046FFF7EC
:10D4500055FE324651460298FEF727FF012805D0B7
:10D460003346029A51465046FEF76AFF2A464CA9B7
:10D470005046FFF7CDFB6DB0BDE8F08F4346224626
:10D48000D8F8A47059465046B84749460CA8FFF74B
:10D49000B5FA4946071C14A818BF0127FFF7AEFAD2
:10D4A000002814BF02200020384308AB53F8207036
:10D4B0002FB32A46394634A8FFF7C7FA079B2A46F6
:10D4C000F9183CA8FFF7C1FA434622463CA934A804
:10D4D000FFF714FE049B009534AA514644A8FFF7B9
:10D4E000EEFB5B4652463CA934A8CDF80080FFF71E
:10D4F000A0FD434644AA21462046FFF7A2FC09F1BD
:10D50000FF390FFA89F995E72046B4E73846B2E7C4
:10D510000398B0E70649074A074B9B1A03DD043B13
:10D52000C858D050FBDCFDF7F1FBFAF79FFF000075
:10D5300060DA0700002C00208C2C0020FEE7FEE7BC
:10D54000FEE7FEE7FEE7FEE7FEE7FEE7FEE7FEE7B3
:10D550009140031C90409C46203A9340194352420C
:10D560006346D3401943704710B5013902449042D5
:10D5700001D1002010BD10F8013B11F8014FA3426A
:10D58000F5D0181B10BD10B5431E0A44914200D1BE
:10D5900010BD11F8014B03F8014FF7E7F8B500BFD4
:10D5A000F8BC08BC9E467047F8B500BFF8BC08BC84
:10D5B0009E467047002C0020011101FF0100000071
:10D5C00000000000021702FE640000000CD60700F5
:10D5D000031704FC04000000ACD6070000000000A4
:10D5E0000000000000000000010100000100000038
:10D5F0000000000002050000210000000000000003
:10D60000000000000000000000000000011104FC08
:10D610000400000000000000021104FC04000000EF
:10D6200000000000032104FC0404000000000000CE
:10D63000041101FF0100000000000000051102FEBE
:10D640000400000000000000061104FC04000000BB
:10D6500000000000071104FC0400000000000000AE
:10D66000081701FF22000000E8D50700091001FF9C
:10D670000100000084D60700000000000000000048
:10D680000000000000000000011704FC7000000012
:10D69000B8D50700021704FCB4000000C4D6070088
:10D6A0000000000000000000000000000101000078
:10D6B0000400000000000000000000000000000066
:10D6C000000000000107000070000000B8D507004E
:10D6D000020100000100000000000000030500003E
:10D6E00041000000000000000000000000000000F9
:10D6F000000000004901B952C5EF41DE27476A55D5
:10D7000027B31CE72D1ECB0FA00C3792BE6AB2E9DF
:10D710009B2403956593690B5EF09CFDA5C02CEEE0
:10D72000F1ECA5A1470A9B3F814C5FD407D8A31415
:10D7300004C609D3F4D60700400000005245414416
:10D740005920544F205550444154450D0A00444936
:10D7500053434F4E4E45435445440D0A00424F4FEC
:10D76000544C4F414445520D0A0052454C454153DB
:10D77000452042544E3120464F52204446550D0A12
:10D78000003C20202020202020202020202020209D
:10D79000202020202020203E0D003D000D0A444680
:10D7A0005520535441525445440D0A0004000000D2
:10D7B0000004010000000402000000040300000057
:10D7C000040400000004050000000406000000043A
:10D7D0000700000004080000000409000000040A1B
:10D7E000000000040B000000140C000000040D00F9
:10D7F0000000040E000000040F00000004100000F0
:10D8000000041100000004120000000413000000D6
:10D8100004140000000415000000041600000004B9
:10D820001700000004180000000419000000041A8A
:10D83000000000041B000000041C240013041D0051
:10D840000003041E000000041F000000982F8A42FD
:10D8500091443771CFFBC0B5A5DBB5E95BC2563942
:10D86000F111F159A4823F92D55E1CAB98AA07D85A
:10D87000015B8312BE853124C37D0C55745DBE727D
:10D88000FEB1DE80A706DC9B74F19BC1C1699BE4FD
:10D890008647BEEFC69DC10FCCA10C246F2CE92D8D
:10D8A000AA84744ADCA9B05CDA88F97652513E98B1
:10D8B0006DC631A8C82703B0C77F59BFF30BE0C6B8
:10D8C0004791A7D55163CA0667292914850AB72746
:10D8D00038211B2EFC6D2C4D130D385354730A65E3
:10D8E000BB0A6A762EC9C281852C7292A1E8BFA2BA
:10D8F0004B661AA8708B4BC2A3516CC719E892D122
:10D90000240699D685350EF470A06A1016C1A419A4
:10D91000086C371E4C774827B5BCB034B30C1C39A3
:10D920004AAAD84E4FCA9C5BF36F2E68EE828F7462
:10D930006F63A5781478C8840802C78CFAFFBE907C
:10D94000EB6C50A4F7A3F9BEF27871C64033002007
:10D950001D33002020000000010000000000000036
:10D9600050EADA308883B89F604F15F30000C98E03
:10D97000001002004466755461726700E8330020AD
:10D9800017BD0700BBBC0700FFC1070071C207003D
:10D9900091C2070005BC0700C9BB070097C107007B
:10D9A0000000000008200001FFFFFFFFFFFFFFFF56
:10D9B000FFFFFFFF0000000000000000000000006B
:10D9C00001000000FFFFFFFF512563FCC2CAB9F34D
:10D9D000849E17A7ADFAE6BCFFFFFFFFFFFFFFFF26
:10D9E00000000000FFFFFFFF96C298D84539A1F460
:10D9F000A033EB2D817D0377F240A463E5E6BCF80C
:10DA000047422CE1F2D1176BF551BF376840B6CBD6
:10DA1000CE5E316B5733CE2B169E0F7C4AEBE78ED2
:10DA20009B7F1AFEE242E34F4B60D2273E3CCE3B47
:10DA3000F6B053CCB0061D65BC86987655BDEBB3E9
:10DA4000E7933AAAD835C65ADDCE070083CE070041
:08DA500065CA07000000000098
:08DA580014AAFF7F0100000089
:10DA600000000000000000000000000000000000B6
:10DA700000000000000000000000000000000000A6
:10DA80000000000000000000000000000000000096
:10DA90000000000000000000000000000000000086
:10DAA0000000000000000000000000000000000076
:10DAB0000000000000000000000000000000000066
:10DAC0000100FFFF0090D0032584070001840700B8
:04DAD0000000000052
:10DAD400001000000030080071B2070000000000D0
:08DAE40049A90700B1A20700E7
:020000020000FC
:020000041000EA
:041014000080070051
:0410180000E00700ED
:040000037000D5159F
:00000001FF
